S02000006F70656E62746C5F6F6C696D65785F73746D3332703130332E7372656307
S315080000004813002001410008E94C0008E94C0008A3
S31508000010E94C0008E94C0008E94C0008E94C0008DE
S31508000020E94C0008E94C0008E94C0008E94C0008CE
S31508000030E94C0008E94C0008E94C0008E94C0008BE
S31508000040E94C0008E94C0008E94C0008E94C0008AE
S31508000050E94C0008E94C0008E94C0008E94C00089E
S31508000060E94C0008E94C0008E94C0008E94C00088E
S31508000070E94C0008E94C0008E94C0008E94C00087E
S31508000080E94C0008E94C0008E94C0008E94C00086E
S31508000090E94C0008E94C0008E94C0008E94C00085E
S315080000A0E94C0008E94C0008E94C0008E94C00084E
S315080000B0E94C0008E94C0008E94C0008E94C00083E
S315080000C0E94C0008E94C0008E94C0008E94C00082E
S315080000D0E94C0008E94C0008E94C0008E94C00081E
S315080000E0E94C0008E94C0008E94C0008E94C00080E
S315080000F0E94C0008E94C0008E94C0008E94C0008FE
S31508000100E94C0008E94C0008E94C0008E94C0008ED
S31508000110E94C0008E94C0008E94C0008E94C0008DD
S31508000120E94C0008E94C0008E94C0008E94C0008CD
S31508000130E94C0008E94C0008E94C0008E94C0008BD
S31508000140E94C0008E94C0008E94C0008E94C0008AD
S31508000150044B9D46C046C046C046C04603F05FF9FC
S3150800016004F000F84813002003E00B780370491CDC
S31508000170401C13005A1E002BF7D1704701E001708E
S31508000180401C13005A1E002BF9D1704710B40023E7
S315080001901400621E002C06D003780C781B1B491C21
S315080001A0401C002BF4D0180010BC704700E0401C1F
S315080001B00278002A02D002788A42F8D1007870477D
S315080001C070B504002079002823D0256B01232A0066
S315080001D014F13401607802F046FA002801D00120B3
S315080001E018E000202071606A854212D3606AE169CE
S315080001F0081885420DD2E67809E0E0694519012319
S315080002002A0014F13401607802F02DFA761E022EC7
S31508000210F3D2002070BD38B504000D00206B85426E
S3150800022012D02000FFF7CCFF002801D001200CE0F7
S3150800023001232A0014F13401607802F0C7F9002876
S3150800024001D0012001E02563002032BD38B5040045
S315080002502000FFF7B5FF0500EDB2002D5DD120782F
S31508000260032852D1607900284FD0002020634FF42C
S315080002700072002114F13400FFF780FF552084F83E
S315080002803202AA2084F83302522084F8340052201D
S3150800029084F83500612084F83600412084F8370058
S315080002A0722084F81802722084F81902412084F812
S315080002B01A02612084F81B02206984F81C0220694E
S315080002C080B2000A84F81D022069000C84F81E0218
S315080002D02069000E84F81F02E06884F82002E068AE
S315080002E080B2000A84F82102E068000C84F8220231
S315080002F0E068000E84F823020123626914F13401D0
S31508000300607802F0B0F90020607100220021607860
S3150800031002F007FA002800D001252800C0B232BD35
S31508000320891E8269921E914201D3002003E08278D9
S31508000330C06A02FB01007047F8B504000D00022DE3
S3150800034002D3A069854201D3012014E02078012850
S3150800035004D00ED303284AD032D30AE02E0016EB77
S315080003605606606A10EB56212000FFF754FF002856
S3150800037002D05FF0FF30F2BD4FF40070B6FBF0F12B
S3150800038001FB1061081990F83470761C606A10EB4E
S3150800039056212000FFF73FFF0028EAD14FF40070EE
S315080003A0B6FBF0F101FB1061081990F8340057EA22
S315080003B00027E80701D5380901E03805000DDAE716
S315080003C0606A10EB15212000FFF725FF0028D0D121
S315080003D068004FF40071B0FBF1F202FB110210192C
S315080003E034304178007850EA012080B2C3E7606A69
S315080003F010EBD5112000FFF70EFF0028B9D1A80091
S315080004004FF40071B0FBF1F202FB110210193430FF
S31508000410C1788278120452EA0161427851EA0221CF
S315080004200078084300010009A5E7F8B504000D00A7
S315080004301600022D02D3A069854201D3022082E06C
S315080004402078012804D07BD3032858D040D377E0FE
S315080004502F0017EB5707606A10EB57212000FFF7AC
S31508000460DAFEC0B200286CD14FF40070B7FBF0F189
S3150800047001FB1071081910F13401E80705D5087851
S3150800048010F00F0050EA061000E0300008707F1CDC
S3150800049001202071606A10EB57212000FFF7BBFE90
S315080004A0C0B200284DD14FF40071B7FBF1F202FB40
S315080004B0117211193431EA0701D5320906E00A78B2
S315080004C012F0F002330A13F00F031A430A7038E0E9
S315080004D0606A10EB15212000FFF79DFEC0B20028C8
S315080004E02FD169004FF40072B1FBF2F303FB12132C
S315080004F0191934310E70B6B2320A4A7021E0606AB0
S3150800050010EBD5112000FFF786FEC0B2002818D1DF
S31508000510A9004FF40072B1FBF2F303FB1213191989
S315080005203431CA78120612F0704216430E70320041
S3150800053092B2120A4A70320C8A70320ECA7000E001
S31508000540022001212171C0B2F2BDF8B504000E00E7
S31508000550022E02D3A069864201D3022527E0002590
S3150800056009E0206910F1010F04D02069401C2061C0
S31508000570012060713E00A069864218D23100200031
S31508000580FFF7DAFE0700002F11D0012F01D102254F
S315080005900DE017F1010F01D1012508E00022310015
S315080005A02000FFF742FF0500EDB2002DD9D0280044
S315080005B0C0B2F2BDF8B504000E00002E07D1E768F8
S315080005C0002F02D0A06987420DD301270BE0310026
S315080005D02000FFF7B1FE022801D2012043E0A169FD
S315080005E0884240D337003D006D1CA069854204D37C
S315080005F00225AF4201D2002035E029002000FFF78E
S315080006009BFE00281DD17FF0704229002000FFF7CD
S315080006100CFFC0B2002806D1002E04D02A003100F3
S315080006202000FFF702FFC0B2002814D1E560206958
S3150800063010F1010F16D02069401E2061012060715B
S3150800064010E010F1010F01D0012800D10BE0BD42E6
S31508000650CAD1002007E0C0B2012802D15FF0FF35F9
S3150800066000E001252800F2BD70B504000D00E58004
S31508000670A068012803D021688969884201D302202D
S3150800068048E0002805D121680978032901D12068A6
S31508000690806A00280ED1E06020680089ADB28542E4
S315080006A001D3022036E02068806AADB210EB15103F
S315080006B0206123E02168897889B20E0100E0AD1B2C
S315080006C0ADB2B6B2B54210D301002068FFF734FECA
S315080006D010F1010F01D101201CE0022803D3216883
S315080006E089698842EBD3022014E0E06001002068A3
S315080006F0FFF716FEADB210EB15102061ADB2102053
S31508000700B5FBF0F101FB1051206810EB41103430B5
S315080007106061002070BDF8B504000D00E088461C35
S31508000720B6B2002E02D02069002801D1042087E045
S31508000730B6B21020B6FBF0F101FB1061002972D1A8
S315080007402069401C2061E068002806D120680089DD
S31508000750B6B2864267D3042072E0B6B220688078C3
S31508000760401E10EA161F5ED1E1682068FFF7E4FD17
S315080007700700022F01D2022062E017F1010F01D112
S3150800078001205DE020688069874246D3002D01D1AB
S31508000790042055E0E1682068FFF70CFF0700002FEA
S315080007A001D107204CE0012F01D1022048E017F1C2
S315080007B0010F01D1012043E02068FFF701FD002861
S315080007C001D001203CE04FF400720021206834304B
S315080007D0FFF7D4FC39002068FFF7A2FD21680863FB
S315080007E0002505E02068006B401C216808636D1C25
S315080007F020688078EDB2854209D22068012101710E
S315080008002068FFF7DDFC0028ECD0012018E02068FE
S31508000810006BEDB2401B21680863E7603900206869
S31508000820FFF77EFD2061E680B6B21020B6FBF0F138
S3150800083001FB1061206810EB411034306061002024
S31508000840F2BD70B504000D0000212000FFF70CFF73
S31508000850C0B200281BD1002621692068FFF7DBFCFF
S31508000860C0B2002813D161690978E52903D0616906
S315080008700978002903D1761CAE4201D107E000268B
S3150800088001212000FFF747FFC0B20028E4D0C0B21C
S3150800089070BDCA7E8B7E53EA022292B20078032884
S315080008A006D1487D097D51EA002080B252EA00420D
S315080008B01000704781760A0092B2120AC2760A0CB4
S315080008C00275090C89B2090A417570472DE9F0418C
S315080008D004000D00287830F04000401E0D2101FB71
S315080008E000F600275FF00108DFF8180D385C40199C
S315080008F04078DFF8101D795C495D51EA00201FFA3F
S3150800090088F8B8F1000F11D080B202F062F880467C
S31508000910FF2E09D234F8160002F05BF8761C1FFA8F
S3150800092088F880B2804508D0002018E080B24FF6DB
S31508000930FF71884201D0002011E07F1C0D2FD3D310
S31508000940287840060AD51FFA88F8B8F1000F05D0AE
S3150800095034F81600002801D0002000E00120BDE888
S31508000960F08170B40A7812F03F02521E0D235A43E2
S3150800097000230124DFF88C5C5D5D6D186D78DFF867
S31508000980846C9E5D765C56EA0525A4B2002C11D0CF
S31508000990FF2A01D3002018E02C0020F81240521C30
S315080009A05B1C0D2BE6D3097849060DD5FF2A08D31B
S315080009B000200AE0ADB24FF6FF76B542F0D000202F
S315080009C003E0002120F81210012070BC7047F0B433
S315080009D04B730F23CB7200230B7300238B760023F4
S315080009E0CB76D2B2531E0D24634300242500A4B24D
S315080009F0ADB24FF6FF76B54202D030F813505B1C05
S31508000A00DFF8006CA65D7554DFF8F86BA65D7618FE
S31508000A10ADB22F0A7770ADB2002D01D14FF6FF7532
S31508000A20641C0D2CE4D3ADB24FF6FF74A54203D077
S31508000A3030F81300002801D152F040020A70F0BCC9
S31508000A4070477CB5040016001D000B222000FFF736
S31508000A508BFBADB2062D09DBADB2E80310EB5500F2
S31508000A6031880D18B61C30880028F5D10720ADB29C
S31508000A70102195FBF1F202FB115212F13001C9B2B5
S31508000A803A2900DBC91D00AA8154401EADB21021C7
S31508000A9095FBF1F5ADB2002DE9D100A97E224254AD
S31508000AA0002100E0491C814202D20A5D202AF9D1C0
S31508000AB00A00511C082803D200ABC35C401C00E0A6
S31508000AC0202313550829F3D373BD00210B22C9B27D
S31508000AD0CB0113EB510103785918401C521E002A0A
S31508000AE0F5D10800C0B270472DE9F0410500002194
S31508000AF02800FFF7B9FD0400E4B2002C02D020005C
S31508000B00C0B226E0FF27B84629692868FFF783FBA5
S31508000B100400E4B2002C1AD16E693078C0B20028FD
S31508000B2001D1042413E0F17A11F03F01C0B2E5289F
S31508000B3004D00A070FD5C9B20F290CD0FF27002108
S31508000B402800FFF7E8FD0400E4B2002CDCD0200002
S31508000B50C0B2BDE8F081C9B20F291ED1E9690029E2
S31508000B60EDD0410606D596F80D8010F0BF000700B7
S31508000B70E9882984C0B2FFB2B8420CD1707B5FFA0B
S31508000B8088F8804507D13100E869FFF79FFE0028FD
S31508000B9001D07F1E00E0FF27D1E7FFB2002F06D164
S31508000BA03000FFF792FF5FFA88F88045CFD0FF271D
S31508000BB04FF6FF702884A869C07AC007BFD40B22F5
S31508000BC0A9693000FFF7E2FA0028B8D1BFE72DE996
S31508000BD0F04104000D00FF26FF275FF00408206996
S31508000BE000282ED021692068FFF715FB80465FFA9A
S31508000BF088F8B8F1000F24D160690278D2B2002AC9
S31508000C0002D15FF004081CE0C17A11F03F01D2B2AC
S31508000C10E52A0BD0D2B22E2A08D0C9B2082901D1AA
S31508000C20012300E00023DBB2AB4215D0FF260021EA
S31508000C302000FFF770FD80465FFA88F8B8F1000FCC
S31508000C40CDD05FFA88F8B8F1000F01D000202061F6
S31508000C504046C0B2BDE8F081C9B20F2919D1510684
S31508000C6005D5477B12F0BF021600E1882184D2B26F
S31508000C70F6B2B2420BD1417BFFB28F4207D10100D7
S31508000C80E069FFF76EFE002801D0761E00E0FF2619
S31508000C90CDE7F6B2002E04D1FFF717FFFFB2874261
S31508000CA002D04FF6FF702084CBE72DE9F04184B0DF
S31508000CB00400A669E7690C22310000A8FFF754FA78
S31508000CC09DF80B00C0072CD50020F0720020E061CB
S31508000CD05FF0010801E018F101081FFA88F8B8F179
S31508000CE0640F0DDA43469BB23A0000A93000FFF7BD
S31508000CF0A8FE2000FFF7F8FE0500EDB2002DEAD0A9
S31508000D001FFA88F8B8F1640F01D107207DE0EDB22B
S31508000D10042D02D02800C0B277E09DF80B00F072CF
S31508000D20E7619DF80B00800712D55FF0000801E027
S31508000D3018F101081FFA88F837F818000028F7D1C3
S31508000D401FFA88F818F119000D2190FBF1F600E05A
S31508000D500126B6B231002000FFF773FD0500EDB29B
S31508000D60002D32D1761E300080B200282DD0E088C2
S31508000D70811B89B22000FFF777FC0500EDB2002D34
S31508000D8023D1A069FFF7A1FE070021692068FFF7B4
S31508000D9042FA0500EDB2002D17D13B00DBB2320056
S31508000DA0D2B26169E069FFF712FE2068012101717C
S31508000DB000212000FFF7AFFC0500EDB2002D04D19D
S31508000DC0761E300080B20028DFD1EDB2002D1AD190
S31508000DD021692068FFF71FFA0500EDB2002D12D130
S31508000DE0202200216069FFF7C9F90B22A169606911
S31508000DF0FFF7BAF9A069C07A10F01800616908739C
S31508000E002068012101712800C0B204B0BDE8F08154
S31508000E1038B50400E588208C4FF6FF71884201D169
S31508000E20290000E0218C89B22000FFF71DFCC0B222
S31508000E3000281BD121692068FFF7EDF9C0B2002808
S31508000E4010D16169E5220A70216801220A71E188D8
S31508000E50ADB2A94206D200212000FFF75CFCC0B261
S31508000E600028E7D0C0B2042800D10220C0B232BDA3
S31508000E702DE9F14F8846D8F8009001E019F10109EB
S31508000E8099F800002F28F9D099F800005C28F5D0C9
S31508000E900098C6690024250002E026F815706D1C26
S31508000EA014F80970641CBFB2202F05DBBFB22F2FC0
S31508000EB002D0BFB25C2F09D114EB0900C8F80000B4
S31508000EC0BFB2202F1FDA5FF004081EE0FF2D01D302
S31508000ED0062090E0FFB20121380080B201F052FDF1
S31508000EE00700BFB2002F01D1062084E0BFB2802FD1
S31508000EF0D3DABFB23900DFF8F808FFF757F9002848
S31508000F00CBD0062077E05FF0000800E06D1E002DCC
S31508000F1009D016EB450030F8027CBFB2202FF5D079
S31508000F20BFB22E2FF2D0002D01D1062063E000209B
S31508000F3026F815000B22202100988069FFF71EF974
S31508000F40002400E0641C36F814002028FAD036F88D
S31508000F5014002E28F6D0002C03D058F0030800E021
S31508000F606D1E002D05D016EB450030F8020C2E2814
S31508000F70F6D15FF00009CB465FF0080A01E058F0A9
S31508000F80030836F81470641CBFB2002F35D10098D8
S31508000F9080690078E52803D10098806905210170E9
S31508000FA0BAF1080F01D15FEA89095FFA89F919F0E0
S31508000FB00C000C2805D05FFA89F919F003000328FC
S31508000FC001D158F002085FEA88700FD45FFA89F9F0
S31508000FD019F00300012801D158F010085FFA89F9C1
S31508000FE019F00C00042801D158F008080098806907
S31508000FF080F80B800020BDE8F28FBFB2202FBED04C
S31508001000BFB22E2F01D1AC42B9D1D34501D2AC42E1
S3150800101013D1BAF10B0F02D158F00308B7E7AC4267
S3150800102001D058F00308A542B1D32C005FF0080B95
S315080010305FF00B0A5FEA8909A3E7BFB2802F10DBCE
S315080010400021380080B201F09DFC0700BFB2002FD6
S3150800105005D0BFB2DFF89C07381810F8807C58F026
S315080010600208BFB2002F07D0BFB23900DFF88807E1
S31508001070FFF79CF8002803D05F2758F003080FE015
S31508001080BFB2B7F141001A2802D259F0020907E0A7
S31508001090BFB2B7F161001A2802D259F00109203F00
S315080010A0009880690BF800701BF1010B69E7F8B529
S315080010B00C0004F209010269002A48D04269137B30
S315080010C000250EE0F6B2052E00D1E5261F0705D548
S315080010D0F6B2B6F141071A2F00D220360E70491C17
S315080010E06D1C082D03D2AE5CF6B2202EEAD1157A15
S315080010F0202D15D02E250D70491C08250AE0DF067F
S3150800110005D5F6B2B6F141071A2F00D220360E7071
S31508001110491C6D1C0B2D03D2AE5CF6B2202EEED107
S31508001120D37A2372D37F957F2D0455EA0363557FBF
S3150800113053EA0523157F2B432360537E157E55EA14
S315080011400323A380D37D927D52EA0322E280002204
S315080011500A70A169002926D0E169002923D0A66969
S315080011600025016900291CD0018C4FF6FF729142B7
S3150800117017D0C76901E0A8556D1C3888BF1C010047
S3150800118089B200290DD0002180B201F0FBFB80B2A4
S31508001190002801D1002504E0E169491E8D42EAD301
S315080011A000250020A855F1BD13B504000198007864
S315080011B02F2803D0019800785C2802D10198401C9A
S315080011C001900020A0600198007820280AD200210A
S315080011D02000FFF749FA0021616120E02068FFF747
S315080011E058FBA06001A92000FFF742FEC0B2002804
S315080011F015D12000FFF778FCA169C97AC0B200288A
S3150800120006D0C0B204280AD1490700D4052006E052
S31508001210490704D46169C87AC006DFD40520C0B27C
S3150800122016BD10B5040001230A0014F134016078D4
S3150800123001F0CCF9002801D003202DE094F8330200
S3150800124094F8321251EA002080B24AF655218842B3
S3150800125001D0022020E094F86C0094F86B10090283
S3150800126051EA004094F86A100843DFF8781C88426F
S3150800127001D1002010E094F8880094F8871009023C
S3150800128051EA004094F886100843DFF8581C884253
S3150800129001D1002000E0012010BDF8B51500026854
S315080012A01378B3F130060A2E05D253783A2B02D1B9
S315080012B0921C026000E0002600200860002E01D083
S315080012C00B209DE1DFF8200C50F82640002C01D1B8
S315080012D00C2095E10C60207800280DD0607801F08C
S315080012E06CF9C10708D4EDB2002D03D0400701D52B
S315080012F00A2085E1002083E100202070667060786E
S3150800130001F0B8F8C10701D5032079E1EDB2002D47
S3150800131003D0400701D50A2072E1002529002000E4
S31508001320FFF77FFF0600F6B2012E1CD10020C0B2DF
S31508001330002800D0401EC0B214EB001000F2F210D4
S31508001340017900290FD0C17A827A120452EA016122
S31508001350427A51EA0221007A50EA01052900200062
S31508001360FFF75FFF0600F6B2032E01D1012047E121
S31508001370F6B2002E01D00D2042E194F8400094F810
S315080013803F1051EA002080B2B0F5007F01D00D2051
S3150800139036E194F84B0094F84A1051EA002080B2DE
S315080013A000280DD194F85B0094F85A10090451EA04
S315080013B0006094F8591050EA012094F85810084330
S315080013C0E06194F84410E170C9B2012904D0C9B2A9
S315080013D0022901D00D2013E1C9B2484394F84110FF
S315080013E0A170C9B2002903D04A1EC9B2114201D060
S315080013F00D2005E194F8461094F8452052EA01219B
S31508001400218121891022B1FBF2F303FB1213002B71
S3150800141001D00D20F4E094F8481094F8472052EAD9
S31508001420012292B2002A0DD194F8571094F856204A
S31508001430120452EA016194F8552051EA022194F8FF
S3150800144054200A4394F8431094F8423053EA012191
S3150800145089B2002901D10D20D2E089B24318268924
S3150800146013EB16139A4201D20D20C9E0D21AA678B8
S31508001470B2FBF6F2002A01D10D20C1E0012640F6A2
S31508001480F677BA4200D302264FF6F677BA4200D369
S315080014900326921CA261256289B24919616259190B
S315080014A0E162F6B2032E16D12089002801D00D205C
S315080014B0A6E094F8630094F86210090451EA006003
S315080014C094F8611050EA012094F860100843A0626D
S315080014D0A069800015E02189002901D10D208FE03F
S315080014E0616A4018A062F6B2022E02D1A0694000D5
S315080014F007E0A06903214843217E11F0010111EBA1
S315080015005000E16900F2FF10B1EB502F01D20D2017
S3150800151076E05FF0FF3020610020E060F6B2032E2F
S3150800152060D10020607194F8650094F8641051EA5F
S31508001530002080B2401960610123626914F1340108
S31508001540607801F043F800284CD194F8330294F8F7
S31508001550321251EA002080B24AF65521884241D11A
S3150800156094F8370094F83610090451EA006094F8A4
S31508001570351050EA012094F834100843DFF8381A79
S3150800158088422FD194F81B0294F81A12090451EADA
S31508001590006094F8191250EA012094F818120843CA
S315080015A0DFF8181A88421DD194F8230294F82212FB
S315080015B0090451EA006094F8211250EA012094F8CF
S315080015C020120843E06094F81F0294F81E120904DA
S315080015D051EA006094F81D1250EA012094F81C1292
S315080015E0084320612670DFF8D8090088401CDFF818
S315080015F0D0190880E0800020206300202071002098
S31508001600F2BD0000B84C000880B500280BD0016870
S31508001610002908D001680978002904D00168C9881A
S315080016208288914201D0092008E00068407800F0DD
S31508001630C4FFC00701D5032000E0002002BDC0B2E8
S31508001640002801D00B2012E0C0B2DFF89C2852F81F
S315080016502020002A01D000231370002901D000227F
S315080016600A70C0B2DFF8802842F8201000207047C0
S315080016702DE9F2438CB004001500002C01D1092095
S31508001680B3E00020206015F01F0515F0FE0200A942
S315080016900CA8FFF702FE0600F6B2002E40F0A38063
S315080016A009A80690DFF81C0907900C9900A8FFF70F
S315080016B07BFD0600059FF6B2002E02D1002F00D151
S315080016C006261C20054258D0F6B2002E0AD0F6B2DD
S315080016D0042E03D100A8FFF7E8FA060055F008051E
S315080016E0059F08E0F87A1121084201D0072602E092
S315080016F0680700D50826F6B2002E4CD128074AD529
S3150800170001F034F9804687F80E80404680B2000A18
S31508001710F8735FEA184038745FEA18607874002036
S31508001720F87200203877002078770020B8770020F4
S31508001730F87739000098FFF7ACF8814600213800A1
S31508001740FFF7B8F8009801210171B9F1000F22D00E
S315080017500098D0F8308049460098FEF7F6FE060055
S31508001760F6B2002E17D10098B9F10101C1604146C1
S315080017700098FEF750FD06000DE0F6B2002E0AD1DD
S31508001780F87AC00601D5042605E0A80703D5F87A35
S31508001790C00700D50726F6B2002E07D1280701D5BF
S315080017A055F020050098006BE0612762F6B2002E1E
S315080017B019D1A57139000098FFF76BF82061F87FF9
S315080017C0B97F090451EA0060797F50EA0120397F20
S315080017D00843E0600020A0600020A0610098206017
S315080017E00098C088A0803000C0B20DB0BDE8F08374
S315080017F0F84C0008744900081C4D00082DE9F0470C
S31508001800050016001F000C00002038602800FFF7AE
S31508001810FBFEC0B2002801D0C0B2E7E0A8790006F6
S3150800182001D50220E2E0A879C00701D40720DDE04F
S31508001830E868A968401AB04229D2060027E0C5F828
S315080018401890A8684FF40071B0FBF1F202FB110280
S31508001850D2F50078464500D2B0464246A8684FF40D
S315080018600071B0FBF1F303FB1103581910F12401C1
S315080018702000FEF779FC18EB0404A86818EB0000B2
S31508001880A860386818EB00003860B6EB0806002E2A
S3150800189000F0AB80A8684FF40071B0FBF1F202FBD0
S315080018A01102002ACDD1A868400A29688978491EFC
S315080018B011EA00085FFA88F8B8F1000F1AD1A8688B
S315080018C0002801D1286903E069692868FEF734FD14
S315080018D0022805D2A87950F08000A871022085E078
S315080018E010F1010F05D1A87950F08000A8710120E8
S315080018F07CE0686169692868FEF712FD8146B9F1DE
S31508001900000F05D1A87950F08000A87102206DE07B
S315080019105FFA88F818EB09095FEA562ABAF1000F48
S3150800192037D0286880785FFA88F81AEB0801884269
S3150800193005D2286880785FFA88F8B0EB080A53461B
S31508001940DBB24A4621002868407800F03FFE0028AE
S3150800195005D0A87950F08000A871012046E0A87942
S31508001960400611D5A869B0EB090050450CD24FF4D2
S31508001970007215F12401A869B0EB09004FF4007351
S3150800198003FB0040FEF7F0FB4FF4007000FB0AF87B
S3150800199071E7A86948453FF452AFA879400613D5C0
S315080019A00123AA6915F124012868407800F05BFE36
S315080019B0002805D0A87950F08000A871012015E00C
S315080019C0A87910F0BF00A87101234A4615F1240131
S315080019D02868407800F0FAFD00283FF430AFA8796F
S315080019E050F08000A871012000E00020BDE8F087D3
S315080019F02DE9F047050016001F000C00002038608E
S31508001A002800FFF701FEC0B2002801D0C0B270E07E
S31508001A10A879000601D502206BE0A879800701D4D1
S31508001A20072066E0E8683018E96888422DD2002663
S31508001A302BE0C5F81890A8684FF40071B0FBF1F2D6
S31508001A4002FB1102D2F50078464500D2B04642465E
S31508001A502100A8684FF40073B0FBF3FC0CFB130CD1
S31508001A601CEB05002430FEF77FFBA87950F04000F8
S31508001A70A87118EB0404A86818EB0000A860386879
S31508001A8018EB00003860B6EB0806002E26D0A868CA
S31508001A904FF40071B0FBF1F202FB1102002ACAD121
S31508001AA0A868400A29688978491E11EA00085FFA79
S31508001AB088F8B8F1000F30D1A868002808D128693D
S31508001AC0002809D100212868FEF774FD286103E083
S31508001AD069692868FEF76EFD00280CD1E868A968D0
S31508001AE0884201D2A868E860A87950F02000A87159
S31508001AF00020BDE8F087012805D1A87950F08000BC
S31508001B00A8710220F5E710F1010F05D1A87950F068
S31508001B108000A8710120ECE76861A879400613D512
S31508001B200123AA6915F124012868407800F09BFD75
S31508001B30002805D0A87950F08000A8710120D8E7C0
S31508001B40A87910F0BF00A87169692868FEF7E8FB54
S31508001B508146B9F1000F05D1A87950F08000A87127
S31508001B600220C6E75FFA88F818EB09095FEA562AE1
S31508001B70BAF1000F38D0286880785FFA88F81AEB2F
S31508001B800801884205D2286880785FFA88F8B0EBA1
S31508001B90080A5346DBB24A4621002868407800F016
S31508001BA062FD002805D0A87950F08000A8710120B0
S31508001BB09FE7A869B0EB0900504510D24FF40072B0
S31508001BC0A869B0EB09004FF4007101FB004115F15B
S31508001BD02400FEF7C9FAA87910F0BF00A8714FF4DF
S31508001BE0007000FB0AF844E7A86948453FF421AFAE
S31508001BF0A868E9688842BFF41CAF01234A4615F174
S31508001C0024012868407800F0E1FC00283FF411AF71
S31508001C10A87950F08000A87101206AE738B5040059
S31508001C202000FFF7F1FCC0B200284AD1A179890645
S31508001C3047D5A07940060FD50123A26914F12401DE
S31508001C402068407800F00FFD002801D0012039E017
S31508001C50A07910F0BF00A071E1692068FEF7DBFAF1
S31508001C60C0B200282DD1256AE87A50F02000E87223
S31508001C70E0682877E06880B2000A6877E068000CB8
S31508001C80A877E068000EE87721692800FEF712FEBB
S31508001C9000F06CFEA875010089B2090AE975010C05
S31508001CA02976000E68760020A8740020E874A079CA
S31508001CB010F0DF00A0712068012101712068FEF78D
S31508001CC0C5FAC0B232BD10B504002000FFF7A6FF62
S31508001CD0C0B2002801D100212160C0B210BD2DE993
S31508001CE0F04104000D002000FFF78EFC0600F6B256
S31508001CF0002E02D03000C0B2CCE0A079000601D593
S31508001D000220C7E0E068A84203D2A079800700D481
S31508001D10E568A0680027A760002D7BD02168897830
S31508001D204FF4007202FB01F8002810D0411EB1FBE7
S31508001D30F8F16A1EB2FBF8F28A4208D3401EB8F1DF
S31508001D4001018843A060A0682D1A606919E020691E
S31508001D50002815D100212068FEF72CFC012805D1A2
S31508001D60A07950F08000A071022093E010F1010FD5
S31508001D7005D1A07950F08000A07101208AE0206189
S31508001D806061002807D145E06061A16818EB010190
S31508001D90A160B5EB0805A84509D2A17989071ED522
S31508001DA001002068FEF706FC00281CD14546A168FC
S31508001DB06918A1604FF40071B5FBF1F202FB1152EC
S31508001DC0002A27D001002068FEF7AAFA0700002F8C
S31508001DD01ED1A07950F08000A07102205AE00100BF
S31508001DE02068FEF7A9FA10F1010F05D1A07950F085
S31508001DF08000A07101204DE0022803D3216889697B
S31508001E008842C1D3A07950F08000A071022041E039
S31508001E1017EB5527A0684FF40071B0FBF1F202FBEF
S31508001E201102002A2AD0A069874227D0A079400645
S31508001E3013D50123A26914F124012068407800F023
S31508001E4012FC002805D0A07950F08000A07101206E
S31508001E5020E0A07910F0BF00A07101233A0014F128
S31508001E6024012068407800F0B1FB002805D0A0794D
S31508001E7050F08000A07101200CE0A761E068A1681D
S31508001E80884205D2A068E060A07950F02000A071D1
S31508001E903000C0B2BDE8F08131B58CB00C0000222C
S31508001EA003A90CA8FFF7F9F90500EDB2002D15D125
S31508001EB000A80990DFF80C010A900C9903A8FFF70F
S31508001EC073F90500EDB2002D08D10898002804D052
S31508001ED0210003A8FFF7EBF800E006252800C0B2AA
S31508001EE00DB030BD46415400340F002071B595B091
S31508001EF0012200A915A8FFF7D0F90400E4B2002CC6
S31508001F0056D109A806902F480790159900A8FFF7FB
S31508001F104BF90400E4B2002C4AD1059D002D01D1ED
S31508001F20062403E0E87AC00700D5072429000098AC
S31508001F30FEF7AFFC0600E4B2002C21D1E87AC00611
S31508001F401ED5022E01D202241AE0242200A90CA8CA
S31508001F50FEF70AF90E9602210CA8FEF785FB040087
S31508001F60E4B2002C0CD100210CA8FEF730FE0400C8
S31508001F70E4B2002C00D10724E4B2042C00D10024DA
S31508001F80E4B2002C14D100A8FEF742FF0400E4B224
S31508001F90002C0DD1002E04D031000098FEF7D5FA9A
S31508001FA00400E4B2002C03D10098FEF74FF90400B0
S31508001FB02000C0B216B070BD5252614172724161C2
S31508001FC03C0F00208C0A00202DE9FC4104000F007C
S31508001FD0904600252600FFE7781E854213DA00ABF7
S31508001FE0012201A94046FFF709FC009801280AD1F9
S31508001FF09DF80400C0B20D28EED03070761C6D1C1A
S31508002000C0B20A28E8D100203070002D00D1002483
S315080020102000BDE8F68130B583B004000D00E4B2B7
S315080020200A2C03D129000D20FFF7F5FF8DF8004093
S31508002030012401AB220000A92800FFF7D9FC01986A
S31508002040A04201D1012001E05FF0FF303EBD70B52E
S3150800205004000D00002601E0641C761C2078002888
S3150800206009D029002078FFF7D6FF10F1010FF3D128
S315080020705FF0FF3000E0300070BD10B450F8041B6C
S3150800208081B102681218001D50F8043BDC0744BFF2
S31508002090A9F10104E31852F8044B43F8044B091F4D
S315080020A0F9D1EBE710BC704710B582B04FF48051F8
S315080020B0DFF8BC0800F010FD4FF40040ADF8000052
S315080020C003208DF8020010208DF8030000A9DFF820
S315080020D0A00800F09DFC4FF40041DFF8940800F0DA
S315080020E0FBFC002413E00221DFF8880800F03AFD23
S315080020F00028F8D0FF21DFF87C0800F021FD012137
S31508002100DFF8700800F02EFD0028F8D0641C0A2CB1
S31508002110E9D34FF40040ADF8000003208DF8020023
S3150800212018208DF8030000A9DFF8440800F070FCB9
S3150800213013BD00B587B00121082000F01DFD01215F
S315080021404FF4804000F028FD4FF48050ADF80000B1
S3150800215010208DF8030003208DF8020000A9DFF88F
S31508002160100800F055FC4FF48051DFF8040800F021
S31508002170B3FC4FF42040ADF8000003208DF80200B0
S3150800218018208DF8030000A9DFF8E40700F040FCEA
S315080021904FF48040ADF8000048208DF8030000A9F0
S315080021A0DFF8CC0700F034FC0020ADF804004FF44B
S315080021B08270ADF806000020ADF808000020ADF8E2
S315080021C00A000020ADF80C004FF40070ADF80E00C0
S315080021D03820ADF810000020ADF812000720ADF841
S315080021E0140001A9DFF88C0700F07CFC0021DFF859
S315080021F0840700F0A9FC0121DFF8780700F092FCBB
S31508002200FFF752FF07B000BD00B585B00021DFF823
S31508002210640700F087FC0020ADF800004FF48270D8
S31508002220ADF802000020ADF804000020ADF8060065
S315080022300020ADF808004FF40070ADF80A00082039
S31508002240ADF80C000020ADF80E000720ADF8100020
S3150800225000A9DFF8200700F045FC0021DFF8140785
S3150800226000F072FC0121DFF80C0700F05BFC05B0FA
S3150800227000BDDFF80407007850F00100DFF8F81613
S315080022800870704780B5C0B2010089B2DFF8E4066D
S3150800229000F056FC0121DFF8DC0600F063FC00289C
S315080022A0F8D0DFF8D00600F04DFCC0B202BD10B57C
S315080022B00400FF20FFF7E6FF207010BD38B500F0D8
S315080022C09DFC10F5FA75FF20FFF7DCFF0400E4B269
S315080022D0FF2C03D000F092FCA842F4D3E4B2FF2C02
S315080022E001D1012000E0002032BD80B54FF48051B5
S315080022F0DFF87C0600F0F0FBFF20FFF7C3FF01BD07
S3150800230080B54FF48051DFF8680600F0E8FBFF203F
S31508002310FFF7B8FFFFF7D2FF002801D0012002E03F
S31508002320FFF7E3FF002002BDF8B504000D0000F03A
S3150800233065FC10F16407FF20FFF7A4FF0600F6B25C
S31508002340FF2E03D100F05AFCB842F4D3F6B2FE2EA3
S3150800235001D0002011E02000FFF7A9FF641C20002F
S31508002360FFF7A5FF641CAD1E002DF4D1FF20FFF773
S3150800237089FFFF20FFF786FF0120F2BD38B504006C
S315080023800D00FFF79BFF002801D1002024E028005C
S31508002390C0B2FFF777FFEDB2FD2D1CD04FF40075E4
S315080023A02078FFF76FFF641C2078FFF76BFF641C2B
S315080023B0AD1E002DF4D1FF20FFF764FFFF20FFF7C5
S315080023C061FFFF20FFF75EFFC0B210F01F0005286F
S315080023D001D0002000E0012032BD38B504000D0010
S315080023E020060AD514F07F0400213720FFF7F5FFF1
S315080023F0C0B2022801DBC0B23BE0FFF776FFFFF769
S315080024007FFF002801D1FF2033E054F04000C0B21E
S31508002410FFF738FF280EC0B2FFF734FF280CC0B20A
S31508002420FFF730FF280AC0B2FFF72CFF2800C0B21A
S31508002430FFF728FF0125E4B2002C00D19525E4B268
S31508002440082C00D187252800C0B2FFF71BFFE4B28D
S315080024500C2C02D1FF20FFF715FF0A25FF20FFF7F6
S3150800246011FF010604D56D1E2900C9B20029F5D150
S31508002470C0B232BD70B582B0C0B2002801D001200A
S315080024809AE0DFF8F4040078800703D5DFF8E8045B
S31508002490007891E0FFF74DFE4FF48051DFF8D00445
S315080024A000F01DFB002500210020FFF796FF0128FC
S315080024B069D100F0A3FB10F57A764FF4D5710820A0
S315080024C0FFF78BFF01283CD1002406E0FF20FFF729
S315080024D0D9FEE4B200A96054641CE4B2042CF5DB0E
S315080024E09DF8020001284ED19DF80300AA284AD17A
S315080024F000F084FBB04206D25FF08041A920FFF7C6
S315080025006CFF0028F4D100F079FBB0423BD20021E1
S315080025103A20FFF762FF002835D1002406E0FF20A5
S31508002520FFF7B0FEE4B200A96054641CE4B2042CC0
S31508002530F5DB9DF80000400601D50C2500E00425D2
S3150800254021E00021A920FFF748FF022802DA022528
S31508002550A92401E00125012400F050FBB04206D26F
S3150800256000212000C0B2FFF738FF0028F4D100F0A0
S3150800257045FBB04206D24FF400711020FFF72DFF3D
S31508002580002800D00025DFF8F403EDB20560FFF758
S31508002590ACFEEDB2002D0AD0DFF8DC03007810F0AF
S315080025A0FE00DFF8D4130870FFF72EFE01E0FFF7F0
S315080025B060FEDFF8C403007876BDC0B2002801D0FB
S315080025C0012002E0DFF8B0030078704738B50C0048
S315080025D011001D00C0B2002802D1EDB2002D01D1B4
S315080025E004203FE0DFF890030078C00701D50320F8
S315080025F038E0DFF888030078000702D44FF400704B
S315080026004143EDB2012D0DD11120FFF7E6FE00285A
S315080026101FD14FF400712000FFF786FE002818D05E
S31508002620002516E01220FFF7D8FE002811D14FF436
S3150800263000712000FFF778FE002806D014F5007414
S315080026406D1E2800C0B20028F1D100210C20FFF72A
S31508002650C4FEFFF74AFEEDB2002D01D0012000E0CE
S315080026600020C0B232BD70B50C0015001E00C0B205
S31508002670002802D1F6B2002E01D1042050E0BE484F
S315080026800078C00701D503204AE0BB480078400718
S3150800269001D5022044E0B9480078000702D44FF477
S315080026A000704543F6B2012E0DD129001820FFF718
S315080026B094FE00282BD1FE212000FFF75FFE00289C
S315080026C025D0002623E0AD48007810F0060F04D088
S315080026D0F6B231009720FFF780FE29001920FFF790
S315080026E07CFE002813D1FC212000FFF747FE0028B6
S315080026F006D014F50074761E3000C0B20028F2D158
S31508002700FD210020FFF73AFE002800D10126FFF739
S31508002710ECFDF6B2002E01D0012000E00020C0B288
S3150800272070BD30B585B014002200C0B2002801D0B3
S31508002730042019E190480078C00701D5032013E169
S315080027400125C9B2002913D0012917D003295ED063
S315080027500A2900F0BB800B2900F0BD800C2900F087
S31508002760C8800D2900F0D3800E2900F0E380F6E03A
S31508002770FFF7C6FD002800D00025F1E0002109205A
S31508002780FFF72BFE002841D1102100A8FFF7CCFD4A
S3150800279000283BD09DF80000C0B28009C0B20128CD
S315080027A00FD19DF809009DF8081010EB01209DF83F
S315080027B0071011F03F0110EB0140401C8002206019
S315080027C023E09DF8050010F00F009DF80A10C9B225
S315080027D010EBD1109DF8091011F0030110EB410020
S315080027E0851C9DF80800C0B28009C0B29DF8071084
S315080027F010EB81009DF8061011F0030110EB812003
S31508002800401CB5F10901884020600025A8E05B4816
S315080028100078400720D500218D20FFF7DEFD00282F
S3150800282053D1FF20FFF72EFD102100A8FFF77CFDEE
S3150800283000284AD0302503E0FF20FFF723FD6D1E50
S31508002840EDB2002DF8D110209DF80A10C9B2090979
S3150800285088402060002538E000210920FFF7BDFDEB
S31508002860002832D1102100A8FFF75EFD00282CD0E1
S3150800287042480078800713D59DF80A0010F03F00FB
S315080028809DF80B10C9B2C909C9B211EB4000401C2A
S315080028909DF80D10C9B28909491E8840206013E0C9
S315080028A09DF80A00C0F38400C0B2401C9DF80B10C6
S315080028B011F003019DF80B20D2B25209D2B212EBE5
S315080028C0C101491C48432060002549E02B4800689F
S315080028D01070002544E000210920FFF77EFD00283E
S315080028E006D110212000FFF71FFD002800D0002583
S315080028F036E000210A20FFF770FD002806D11021D6
S315080029002000FFF711FD002800D0002528E000214F
S315080029103A20FFF762FD00280BD1002505E0FF20CD
S31508002920FFF7B0FCEDB228556D1CEDB2042DF6DBB1
S31508002930002515E01148007840070FD500218D20A5
S31508002940FFF74BFD002809D1FF20FFF79BFC40212C
S315080029502000FFF7E9FC002800D0002500E0042548
S31508002960FFF7C3FC2800C0B205B030BD0448704765
S31508002970000C01400038004000000020380F0020FD
S315080029800000AA4280B2802801DA01001EE0002970
S315080029900CD080B2FF2801DD002106E080B219497B
S315080029A011EB4000B0F5807001880FE0002100E0CF
S315080029B0491C89B2802906DA89B2124A32F81120EE
S315080029C080B29042F4D111F18000C1B2080080B201
S315080029D07047002100E0491C0B4A32F81120002AF2
S315080029E005D0094A32F8112080B29042F3D1064A3E
S315080029F032F81120002A03D0044830F81100FFE706
S31508002A0080B27047D847000818440008F8450008FF
S31508002A10F0B400220026002400250023002791F8A0
S31508002A2003C01CF00F0C624691F803C05FEACC6C39
S31508002A3001D58B781A430B781B0621D0036800242E
S31508002A4006E0CD78482D02D10125A5400561641C14
S31508002A50082C14D20125A5400E882E40AE42F6D188
S31508002A60A5000F2616FA05F7BB4312FA05F52B4300
S31508002A70CD78282DE5D10125A5404561E7E7036016
S31508002A800B88FF2B26DD4368002420E0012514F17E
S31508002A900806B5400E882E40AE4217D1A5000F266F
S31508002AA016FA05F7BB4312FA05F52B43CD78282D00
S31508002AB004D1012514F10806B5404561CD78482DA5
S31508002AC004D1012514F10806B5400561641C082CDB
S31508002AD0DCD34360F0BC704789B20161704789B2A4
S31508002AE04161704710B4002203881A0012F441525B
S31508002AF00B884C8823438C882343CC8823430C8932
S31508002B0023434C8923438C892343CC8923431A4383
S31508002B100280828B4FF2FF731A408283098A0182F0
S31508002B2010BC7047C9B2002904D0018851F0400191
S31508002B30018004E001884FF6BF721140018070479A
S31508002B408181704780897047C9B2002904D00188FD
S31508002B5051F40051018004E001884DF6FF721140DE
S31508002B600180704700220089084201D0012200E056
S31508002B7000221000C0B27047C9B2002905D00E491C
S31508002B80096808430C49086005E00B49096831EAF9
S31508002B900000094908607047C9B2002905D00749ED
S31508002BA0096808430549086005E00449096831EAE7
S31508002BB00000024908607047181002401C100240C5
S31508002BC080B500F00DF81048104901601048002142
S31508002BD001601048052101600F480021018001BDF0
S31508002BE00C480021016070470A480068C00304D5F4
S31508002BF009480088401C08490880704780B5FFF7D7
S31508002C00F3FF0548008802BD14E000E03F19010003
S31508002C1018E000E010E000E03E0F002080B5DFF885
S31508002C20780600210170DFF874160020FEF707FD0C
S31508002C30C0B2002804D09121DFF8640600F0C0FB7A
S31508002C4001BDDFF854060078002801D1012000E014
S31508002C500020704780B500F0F1FB012801D1002063
S31508002C6011E0DFF834060078002801D000200AE0D9
S31508002C7000F0E8FB012805D1DFF81C0601210170E8
S31508002C80012000E0002002BD10B5DFF80C06007830
S31508002C90002800F0FF81DFF800060078012834D10B
S31508002CA000F0EAFBDFF8FC0500F014FCDFF8F80595
S31508002CB000F010FC00F0DEFB01220100DFF8EC0555
S31508002CC0FEF7D6FC002807D0DFF8E40500F002FC82
S31508002CD0012000F0F5FBDDE1DFF8D80500F0FAFB8E
S31508002CE0DFF8D40500F0F6FBDFF8D00500F0F2FBBC
S31508002CF0DFF8CC0500210160DFF8C405002141603A
S31508002D00DFF8940502210170C4E1DFF88C0500782C
S31508002D10022840F0F780DFF894254FF48071DFF839
S31508002D20A405FFF751F9DFF8741591F83A12C1F3C3
S31508002D30C01111F0010101290FDBDFF8740500F05D
S31508002D40C9FB022000F0BCFBDFF86005FEF7BBFFFD
S31508002D50DFF84405002101709CE100281BD0002201
S31508002D60DFF86415DFF85C0500F0D6F9040024B234
S31508002D7014F1010F0FD1DFF8380500F0ABFB032083
S31508002D8000F09EFBDFF82405FEF79DFFDFF8080537
S31508002D90002101707EE124B2012C28DBDFF8200532
S31508002DA0406800280BD1DFF81C05D0F88001DFF851
S31508002DB010150860DFF8080524B2446017E0DFF84C
S31508002DC00405D0F88001DFF8F8140968884206D2AD
S31508002DD0DFF8F004D0F88001DFF8E4140860DFF8C3
S31508002DE0E004406824B22018DFF8D4144860DFF8FD
S31508002DF0AC04D0F83C02DFF8A414D1F8401288429B
S31508002E0001D1012000E000200128C0F24381002101
S31508002E10DFF89804FEF763FF00280FD0DFF8900468
S31508002E2000F058FB042000F04BFBDFF88004FEF7A7
S31508002E304AFFDFF86404002101702BE1DFF874040F
S31508002E4000F048FBDFF8840400F044FBDFF8801448
S31508002E50DFF86C04406800F075FADFF8740400F0D7
S31508002E6039FBDFF8700400F035FBDFF86414DFF88F
S31508002E7050040068000EC0B200F053FADFF8581488
S31508002E80DFF83C040068000CC0B200F04AFADFF82C
S31508002E904C14DFF82C040068000AC0B200F041FAAE
S31508002EA0DFF83C14DFF818040068C0B200F039FAFD
S31508002EB0DFF81C0400F00EFB77A000F00BFBDFF830
S31508002EC000044168DFF8F803006800F039FB0028C1
S31508002ED00FD1DFF8DC0300F0FDFA052000F0F0FA68
S31508002EE0DFF8C803FEF7EFFEDFF8AC030021017038
S31508002EF0D0E0DFF8C00300F0EDFADFF89C03032109
S31508002F000170C7E0DFF890030078032840F0C2801C
S31508002F10DFF898234FF48071DFF8A803FFF754F819
S31508002F20DFF8781391F83A12C1F3C01111F00101D4
S31508002F3001290EDBDFF8AC0300F0CCFA022000F022
S31508002F40BFFADFF86803FEF7BEFED348002101701A
S31508002F50A0E000281AD0DFF89023DFF86C13DFF81A
S31508002F60640300F0D9F8040024B214F1010F0DD15E
S31508002F70DFF8780300F0AEFA032000F0A1FACB4898
S31508002F80FEF7A1FEC4480021017083E024B2012C9B
S31508002F904CDBD74800F09EFACD4924B2200000F059
S31508002FA0D1F9CB4800F096FAD24800F093FAC8490E
S31508002FB0C448D0F88001000EC0B200F0B2F9C64984
S31508002FC0C048D0F88001000CC0B200F0AAF9C34985
S31508002FD0BC48D0F88001000AC0B200F0A2F9C04986
S31508002FE0B848D0F88001C0B200F09BF9B84800F0A4
S31508002FF071FA29A000F06EFABB4A24B22100B14842
S31508003000D0F8800100F098FA00280CD1A84800F002
S3150800301061FA062000F054FAA448FEF754FE9E48CA
S315080030200021017036E0A34800F054FA9B48D0F816
S315080030303C029A49D1F84012884201D1012000E0A9
S315080030400020012826DBAC4800F044FA00F080FA9C
S3150800305000280CD1964800F03DFA072000F030FA17
S315080030609248FEF730FE8C480021017012E0914824
S3150800307000F030FAA14800F02DFA8C48FEF723FE3E
S315080030809F4800F027FA84480021017000F005FAED
S3150800309000F068FA10BD00002E2E2E0010B50400B0
S315080030A0207800F08AFA532804D1607800F089FA6B
S315080030B0002801D103200FE06078312801D10020D3
S315080030C00AE06078322801D1012005E060783328CB
S315080030D001D1022000E0032010BD70B504000026CF
S315080030E0A41C200000F047F90500AE19A41C200016
S315080030F000F041F986196D1EA41CADB2022DF6DA50
S31508003100F6B2F643200000F036F9F6B2864201D050
S31508003110002000E0012070BD2DE9F04105000E00F9
S3150800312014005FF00008002E01D0002D04D14FF4E2
S3150800313015715B4800F044F92800FFF7AFFF070058
S31508003140FFB2032F01D10020A3E02800FFF7C5FF37
S31508003150002802D15FF0FF309BE0FFB2002F03D0BA
S31508003160022F5AD028D392E0AD1C280000F003F9AC
S315080031700700AD1C280000F0FEF800023060AD1C08
S31508003180D6F80080280000F0F6F810EB080030604A
S31508003190AD1CB7F10308002C0DD0002606E0280068
S315080031A000F0E9F8B6B23055AD1C761CB6B20FFA87
S315080031B088F84645F3DB6AE0AD1C280000F0DBF82A
S315080031C00700AD1C280000F0D6F800043060AD1CDE
S315080031D0D6F80080280000F0CEF818EB0020306002
S315080031E0AD1CD6F80080280000F0C5F810EB0800E2
S315080031F03060AD1CB7F10408002C0DD0002606E09F
S31508003200280000F0B8F8B6B23055AD1C761CB6B238
S315080032100FFA88F84645F3DB39E0AD1C280000F0C4
S31508003220AAF80700AD1C280000F0A5F800063060D3
S31508003230AD1CD6F80080280000F09DF818EB004079
S315080032403060AD1CD6F80080280000F094F818EB22
S3150800325000203060AD1CD6F80080280000F08BF8FE
S3150800326010EB08003060AD1CB7F10508002C0DD036
S31508003270002606E0280000F07EF8B6B23055AD1CF0
S31508003280761CB6B20FFA88F84645F3DBFFE74046E8
S3150800329000B2BDE8F0810000410F002004000020C4
S315080032A0C84A00087C4B0008544B00083802002026
S315080032B0244D00082C4D0008A04B0008F84A0008C9
S315080032C0200F00208C0C00200C0E0020044D000856
S315080032D0E00E0020504C0008E20E0020E40E00200C
S315080032E0E60E0020C44B00088C0D0020E84B0008B1
S315080032F0C84C0008884C00086C4C0008A04C000814
S31508003300284B000880B5010011F00F003030C9B213
S315080033100A2901DBC01D02E0C0B200F04EF9C0B2B6
S3150800332002BD38B504000D00E4B22009FFF7EAFF34
S31508003330287014F00F00FFF7E5FF68700020A870EA
S31508003340280032BD0200491C0A23B2FBF3F2002A08
S31508003350F9D100220A700200491E0A20B2FBF0F3D6
S3150800336000FB1320303008700A20B2FBF0F2002A66
S31508003370F2D10800704770B504000025002609E060
S315080033803038C0B20A2800DBC01FEDB2C0B210EB5D
S315080033900515761CF6B2022E0FDAF6B2305D00F08D
S315080033A00CF9C0B2B0F13001172904D2C0B2B0F19D
S315080033B03A010729E4D2002001E02800C0B270BD16
S315080033C080B5034A10600348016000F003F9FCE782
S315080033D0280F00202C0F002080B515480088ADF86E
S315080033E0000000F009F900F033FB124800780128C4
S315080033F002D100A800F02AF901BD80B50E4800F0F8
S315080034006DFB012802D10C4800F020F901BD704778
S3150800341080B5C9B200F038FB00F012F901BD0548C5
S3150800342001210170704703480021017070470000B0
S315080034304E3A0008440F0020A00E002080B500F088
S31508003440F6F802BD00B589B000A8202100F0B0FB4F
S3150800345000A93348FEF720FD002808D10098002867
S3150800346005D09DF80800C00601D4012000E0002020
S3150800347009B000BD2A48704780B52A48002180F85F
S3150800348024120A2228492748FEF7F2F8002803D111
S315080034902448012180F8241201BD80B5214890F8FE
S315080034A02402012802D11F48FEF70DFC40211F48BF
S315080034B000F086FB0028F9D01948FEF717FD01BD74
S315080034C080B5184890F82402012802D11548FEF75D
S315080034D0FAFB01BD10B50400124890F82402012831
S315080034E019D110492000FEF7B2FD002813D50D4862
S315080034F0002180F824120B48FEF7E5FB0BE0217843
S3150800350089B20A4800F058FB8021084800F058FBA9
S315080035100028F9D0641C20780028F0D110BD0000DE
S31508003520304C00085C040020D84C000800440040D9
S3150800353080B500F053FB01BD80B500F05AFB02BD13
S3150800354080B500F082FB02BD80B500F0DDFB02BD50
S3150800355080B500F094FB002801D1002001E000F0BE
S3150800356004FC02BD80B5FFF7EFFF00280AD0FFF77D
S315080035704EFFFFF735FB04484FF4C041016003488E
S315080035800068804701BD000008ED00E004600008FF
S3150800359070B504000D00160005E0287820706D1C33
S315080035A0641C00F017F83000461E80B20028F4D1DB
S315080035B070BD80B500F0A4FD01BD80B500F0ACFD7E
S315080035C002BD30380A2801D2012000E00020C0B22E
S315080035D070477047704750F8041B61B150F8042BC8
S315080035E0D30744BFA9F101039A18002342F8043B04
S315080035F0091FFAD1EFE77047DFF83404002101709C
S31508003600DFF82C0400218164DFF82404002180F807
S315080036104310DFF81C040021A0F84410DFF810045A
S3150800362000218170DFF80804002141707047DFF837
S3150800363000040078002801D1002000E0012070472E
S31508003640DFF8EC03002180F84310704780B5017855
S31508003650FF2918D100F08BF8DFF8D40390F843005F
S31508003660012802D1102000F078F8DFF8C403012100
S3150800367080F84310DFF8B803B0F94410DFF8B40354
S3150800368000F053F801BDDFF8A813097801294BD1DA
S315080036900178C92932D0CC293FD0CF293AD0D029B0
S315080036A02FD0D12933D0D2292ED0F32917D0F429F7
S315080036B00FD0F5290AD0F6290ED0FA2912D0FC29FE
S315080036C013D0FD2914D0FE2915D029E000F0D5F82D
S315080036D0C2E700F0F1F8BFE700F0C4F8BCE700F075
S315080036E00DF9B9E700F0A6F8B6E700F09DF8B3E7DC
S315080036F000F082F8B0E700F070F8ADE700F02FF9B7
S31508003700AAE700F046F9A7E700F00FF9A4E700F0EA
S315080037106EF9A1E700F07FF99EE700F093F99BE7C1
S31508003720202000F01AF897E7ACE780B589B2FFF7D2
S315080037306FFE01BD10B4002302E00478E318401CB4
S315080037400C00611E002CF8D1DBB21360012010BCFE
S315080037507047B748002141707047B549FE22CA70C4
S31508003760B3490871B2480221A0F84410704710B551
S315080037700400FFF766FA002803D11020FFF7EDFFD3
S315080037802AE0FFF7E6FFAA4801210170A848FF21B1
S31508003790C170A74800210171A548007950F01000B2
S315080037A0A3490871A24800214171A148A049497955
S315080037B041719F48402181719D484021C1719C48B3
S315080037C0002101729A4801214172994801218172AA
S315080037D097480821A0F8441010BD10B50400944875
S315080037E000210170FFF7B5FF9148FF21C17090488D
S315080037F00121A0F8441010BD8D49FF22CA708C49DA
S3150800380000220A718A498A4A52784A7188490022EE
S315080038108A7187490022CA71854900220A72844939
S315080038200622A1F84420704710B504000020FFF7CF
S3150800383094FF10BD7E49FF22CA707D497E4A8A647C
S315080038407B4900220A717A4900224A717849002286
S315080038508A7177490722C1F8072075490822A1F815
S31508003860442070477249FF22CA70714940688864CB
S315080038706F480121A0F84410704710B5040060781D
S31508003880402803DB2220FFF768FF14E0627892B233
S315080038906748816C6948FFF77BFE6548FF21C17060
S315080038A06348806C61780818614988646078401CB0
S315080038B05F49A1F8440010BD10B50400607840289F
S315080038C003DB2220FFF749FF17E059486168816446
S315080038D0627892B25648816C5848FFF759FE5448A8
S315080038E0FF21C1705248806C617808185049886475
S315080038F06078401C4E49A1F8440010BD80B54C497B
S31508003900FF22CA704E4A41684948806CFFF712FF89
S31508003910474908714648002141714548002181718F
S3150800392043480821A0F8441001BD4149FF22CA7046
S315080039303F4900220A713E4900224A713C49402209
S315080039408A713B490022CA71394900220A723849EC
S3150800395000224A7236490722A1F84420704780B5EA
S31508003960421C3F213248806CFFF7E6FD002803D150
S315080039703120FFF7F2FE0BE02D48FF21C1702C48DD
S31508003980806C3F302A49886429480121A0F84410F0
S3150800399001BD10B5040060783F2803DB2220FFF73D
S315080039A0DCFE23E02248FF21C17021480121A0F84E
S315080039B044106078002807D1FFF7CAFD002802D115
S315080039C03120FFF7CAFE11E0A21C61781848806C06
S315080039D0FFF7B2FD002803D13120FFF7BEFE05E050
S315080039E01348806C617808181149886410BD80B541
S315080039F041680F48806CFFF7A3FD002803D13120EA
S31508003A00FFF7ABFE06E00A48FF21C170084801210E
S31508003A10A0F8441001BD10B50400FFF7CAFD04481C
S31508003A20FF21C17002480121A0F8441010BD000012
S31508003A30100E0020130E0020344D0008140E00202E
S31508003A40170E002080B53120FFF787FE01BDFF0065
S31508003A504B48002101804B48002101804A4800213B
S31508003A6001804A48002101804948002101804448D4
S31508003A7040F2712101804348008840F4005050F01C
S31508003A800C0040490880704770B504000D00EDB27F
S31508003A90412D03DB88213F48FFF792FC2800C0B27E
S31508003AA000F05AF8012803D08B213A48FFF788FC22
S31508003AB000260CE0FFF78EFDB6B2305D00F04CF83C
S31508003AC0012803D093213348FFF77AFC761C280097
S31508003AD0C0B2B6B280B28642ECD370BD10B504004F
S31508003AE02D48007800280CD12C4800F02AF8012827
S31508003AF005D12948012101702948002101700020BB
S31508003B0010BD2748007825494018401C00F019F8D0
S31508003B100128F4D122480078401C21490870204821
S31508003B2000781E4909788842E9D11D48027892B280
S31508003B301C492000FFF72CFD1748002101700120C1
S31508003B40DEE719490988890604D5184909880170E4
S31508003B50012000E00020704780B51349098809064E
S31508003B6001D400200AE01149C0B2088001E0FFF73D
S31508003B7031FD0D4800880006F9D5012002BD000078
S31508003B80084400400C4400401044004014440040DF
S31508003B90184400408C4A0008430F00205C0E0020A1
S31508003BA0420F00205D0E00200044004004440040FF
S31508003BB0002200F0BDBA0000C905C90D8180704712
S31508003BC0002289B2B1F5007F0088084201D001229F
S31508003BD000E000221000C0B270470000DFF8FC04C5
S31508003BE05FF0FF310160DFF8F8045FF0FF31016034
S31508003BF0704770B504000D001600200000F00AFAA0
S31508003C00FF2805D02819401E00F004FAFF2801D124
S31508003C10002019E0600A4FF400714843DFF8C41425
S31508003C200968884208D12B009BB232002100DFF8D0
S31508003C30B00400F0F1F807E02B009BB23200210037
S31508003C40DFF8980400F0E8F870BD70B504000D00C0
S31508003C50200000F0DFF906002819401E00F0DAF906
S31508003C60F6B2FF2E02D0C0B2FF2801D1002005E02F
S31508003C700100C9B23000C0B200F05DF970BD80B570
S31508003C8000200090DFF85804006810F1010F01D1F8
S31508003C90012038E00098DFF84814496808180090B1
S31508003CA00098DFF83C148968081800900098DFF837
S31508003CB03014C968081800900098DFF824140969B8
S31508003CC0081800900098DFF8181449690818009039
S31508003CD00098DFF80C148969081800900098DFF836
S31508003CE00014C969081800900098C043009000980D
S31508003CF0401C009000AA0421DFF8E803006810F5CC
S31508003D00A870FFF776FF02BD0020DFF8D813096810
S31508003D1009680818DFF8CC13096849680818DFF835
S31508003D20C413096889680818DFF8B8130968C968E8
S31508003D300818DFF8B013096809690818DFF8A4132A
S31508003D40096849690818DFF89C1309688969081819
S31508003D50DFF89013096811F5A87109680818002892
S31508003D6001D1012000E00020704780B5DFF870031C
S31508003D70006810F1010F07D0DFF8640300F090F82F
S31508003D80002801D100200EE0DFF85003006810F18A
S31508003D90010F07D0DFF8440300F082F8002801D1AC
S31508003DA0002000E0012002BD80B54FF40072B1FB8F
S31508003DB0F2F303FB1213002B01D000200BE002687C
S31508003DC08A4201D1012006E001604FF40072001D0D
S31508003DD0FFF7DEFB012002BD38B504000D00C04820
S31508003DE0844208D1BD4C29002000FFF7DDFF0028DA
S31508003DF010D100200FE0BB480068854203D1B84CBB
S31508003E00B8480568EFE7200000F04AF80028EAD12C
S31508003E10002000E0200032BD2DE9F04104000F002B
S31508003E2015001E00780A4FF4007101FB00F820689F
S31508003E3010F1010F07D141462000FFF7B5FF002812
S31508003E4001D100202AE02068404508D041462000DC
S31508003E50FFF7C2FF0400002C01D100201EE02068F5
S31508003E60381A0019071DFFF7B5FB201D381AB0F5DB
S31508003E70007F0AD318F500712000FFF7ADFF040094
S31508003E80002C01D1002009E0271D287838707F1CF6
S31508003E906D1C761EB6B2002EE5D10120BDE8F08174
S31508003EA02DE9F04104000125206800F0B3F8C0B2FE
S31508003EB0FF2801D100203CE000F09BF88A48006802
S31508003EC0C00703D500F09FF8002032E08748006855
S31508003ED050F0010085490860002600E0761C802E17
S31508003EE01DD2206810EB860714EB8600D0F80480F4
S31508003EF0A7F8008001E0FFF76DFB7B480068C00764
S31508003F00F9D45FEA1840788001E0FFF763FB76484A
S31508003F100068C007F9D438684045DFD000257348E3
S31508003F200068400840007149086000F06CF82800F5
S31508003F30C0B2BDE8F08170B505000C00E4B2EDB280
S31508003F40AC4201D2002053E06648007AEDB28542C1
S31508003F5005D3644890F89800E4B2A04201D2002044
S31508003F6046E000F046F860480068C00703D500F050
S31508003F704AF800203CE05D48006850F002005B49C2
S31508003F8008602800C0B200F06FF805002000C0B233
S31508003F9000F06AF806002000C0B200F082F8801926
S31508003FA0401E401B401C840A002606E0FFF712FB51
S31508003FB04D480068C007F9D4761CB6B2A4B2A6422A
S31508003FC00DD2B6B24FF4806000FB0650484908602F
S31508003FD04648006850F0400044490860E8E743480E
S31508003FE0006830F002004149086000F00CF8012032
S31508003FF070BD4048404901603E48404901603A4822
S315080040003421016070473948006850F0800037490C
S315080040100860704738B50400002500E06D1CEDB255
S315080040200D2D1FD2FFF7D6FAEDB20C202D4900FB55
S31508004030051000688442F1D3EDB20C20294900FB33
S3150800404005100068EDB20C21264A01FB05214968D6
S3150800405008188442E2D2EDB20C20224900FB051072
S31508004060007A00E0FF2032BD38B50400002500E0E4
S315080040706D1CEDB20D2D11D2FFF7ACFAEDB20C2086
S31508004080184900FB0510007AE4B2A042F0D1EDB25F
S315080040900C20144900FB0510006801E05FF0FF30B2
S315080040A032BD38B50400002500E06D1CEDB20D2DBB
S315080040B011D2FFF78FFAEDB20C200A4900FB051062
S315080040C0007AE4B2A042F0D1EDB20C20054900FB1B
S315080040D00510406800E0002032BD0000840600207C
S315080040E088080020D84800080C200240102002400A
S315080040F0142002400420024023016745AB89EFCD16
S31508004100044B9D46C046C046C046C046FFF78BF9DD
S3150800411000F028F84813002010B50400200000F02D
S315080041202CF8002801D0203CFFE7200010BD000035
S3150800413000B500BF130096469446103928BFA0E87C
S315080041400C50FAD85FEA417C28BF0CC048BF40F83B
S31508004150042BC90728BF20F8022B48BF00F8012BFB
S3150800416000BD000000F011F8002801D000F010F89A
S31508004170002000F021F800F0F5F861381A2801D27D
S31508004180012000E00020C0B27047012070470000FF
S3150800419010B5074979441831064C7C44163404E0B6
S315080041A00A68081D511888470146A142F8D110BD72
S315080041B05C0A00007C0A000080B500F005F800F0F3
S315080041C0D3F800F0DFF8FCE700B583B000200090D4
S315080041D0002001905948006850F0010057490860CE
S315080041E057480068574908405549086053480068C9
S315080041F055490840514908605048006830F4802005
S315080042004E4908604E48006830F4FE004C49086084
S315080042104E485FF41F0101604848006850F480303A
S31508004220464908604548006810F400300190009837
S31508004230401C00900198002804D1009840F2DC51F7
S315080042408842EFD13D480068800303D47321404873
S31508004250FFF7B6F83F48006850F010003D4908607F
S315080042603C480068800880003A4908603948006878
S3150800427050F0020037490860314831490968016041
S315080042802F48006850F400502D4908602C480068F3
S3150800429050F480602A4908602948006830F47C1088
S315080042A0274908600920801E80042549096850F4BA
S315080042B080300843224908602048006850F0807022
S315080042C01E4908601D4800688001FBD51C48006827
S315080042D0800880001A4908601948006850F00200F2
S315080042E0174908601648006810F00C000828F9D12C
S315080042F01948006850F400301749086017480068E4
S3150800430050F00500154908601548006830F47060DB
S31508004310134908601248006850F430601049086074
S315080043200F48006830F470400D4908600C48006872
S3150800433050F480400A49086007BD0000001002409A
S31508004340041002400000FFF8FFFFF6FE08100240C6
S31508004350F4490008002002401C10024018100240D0
S315080043600008014000F01AB880B5FFF732F9FEF7E9
S3150800437027FCFFF7DDF8FEF751FCFFF72DF800F0F4
S3150800438013F801BD80B5FFF725F9FEF72DFCFEF7FA
S315080043907BFCFFF732F800F012F801BD07463846F5
S315080043A000F030F8FBE7000080B5144801210170E1
S315080043B0FEF724FC1249086000F001F801BD80B53B
S315080043C0FFF73CF8012817D0FEF73BFC002813D06E
S315080043D00A48007801280FD1FEF710FC0849096839
S315080043E03231884208D3054800210170FEF732FCB5
S315080043F0002801D1FFF7B6F801BD0000400F0020E4
S31508004400300F002080B5C046C046024A1100182069
S31508004410ABBEFBE726000200610062006300640091
S31508004420650066006700680069006A006B006C003A
S315080044306D006E006F0070007100720073007400EA
S31508004440750076007700780079007A00A100A2004E
S31508004450A300A500AC00AF00E000E100E200E30025
S31508004460E400E500E600E700E800E900EA00EB0002
S31508004470EC00ED00EE00EF00F000F100F200F300B2
S31508004480F400F500F600F800F900FA00FB00FC005D
S31508004490FD00FE00FF0001010301050107010901F6
S315080044A00B010D010F011101130115011701190166
S315080044B01B011D011F0121012301250127012901D6
S315080044C02B012D012F0131013301350137013A0145
S315080044D03C013E01400142014401460148014B01AD
S315080044E04D014F01510153015501570159015B0116
S315080044F05D015F01610163016501670169016B0186
S315080045006D016F0171017301750177017A017C01F3
S315080045107E019201B103B203B303B403B503B60334
S31508004520B703B803B903BA03BB03BC03BD03BE0391
S31508004530BF03C003C103C303C403C503C603C7033C
S31508004540C803C903CA0330043104320433043404EB
S31508004550350436043704380439043A043B043C0469
S315080045603D043E043F044004410442044304440419
S31508004570450446044704480449044A044B044C04C9
S315080045804D044E044F045104520453045404550474
S3150800459056045704580459045A045B045C045E0420
S315080045A05F0470217121722173217421752176218E
S315080045B07721782179217A217B217C217D217E2111
S315080045C07F2141FF42FF43FF44FF45FF46FF47FF68
S315080045D048FF49FF4AFF4BFF4CFF4DFF4EFF4FFF79
S315080045E050FF51FF52FF53FF54FF55FF56FF57FF29
S315080045F058FF59FF5AFF000041004200430044009B
S31508004600450046004700480049004A004B004C0058
S315080046104D004E004F005000510052005300540008
S31508004620550056005700580059005A002100E0FF6F
S31508004630E1FFE5FFE2FFE3FFC000C100C200C300DF
S31508004640C400C500C600C700C800C900CA00CB0020
S31508004650CC00CD00CE00CF00D000D100D200D300D0
S31508004660D400D500D600D800D900DA00DB00DC007B
S31508004670DD00DE00780100010201040106010801DF
S315080046800A010C010E01100112011401160118018C
S315080046901A011C011E0120012201240126012801FC
S315080046A02A012C012E01300132013401360139016B
S315080046B03B013D013F0141014301450147014A01D3
S315080046C04C014E01500152015401560158015A013C
S315080046D05C015E01600162016401660168016A01AC
S315080046E06C016E01700172017401760179017B011A
S315080046F07D01910191039203930394039503960315
S315080047009703980399039A039B039C039D039E03AF
S315080047109F03A003A103A303A403A503A603A7035A
S31508004720A803A903AA031004110412041304140409
S31508004730150416041704180419041A041B041C0487
S315080047401D041E041F042004210422042304240437
S31508004750250426042704280429042A042B042C04E7
S315080047602D042E042F040104020403040404050482
S3150800477006040704080409040A040B040C040E04BE
S315080047800F0460216121622163216421652166216C
S315080047906721682169216A216B216C216D216E21AF
S315080047A06F2121FF22FF23FF24FF25FF26FF27FF76
S315080047B028FF29FF2AFF2BFF2CFF2DFF2EFF2FFF97
S315080047C030FF31FF32FF33FF34FF35FF36FF37FF47
S315080047D038FF39FF3AFF0000C700FC00E900E20095
S315080047E0E400E000E500E700EA00EB00E800EF007F
S315080047F0EE00EC00C400C500C900E600C600F400DF
S31508004800F600F200FB00F900FF00D600DC00A2006B
S31508004810A300A500A7209201E100ED00F300FA002D
S31508004820F100D100AA00BA00BF001023AC00BD00F9
S31508004830BC00A100AB00BB0091259225932502255B
S315080048402425612562255625552563255125572595
S315080048505D255C255B251025142534252C251C256E
S3150800486000253C255E255F255A255425692566259C
S31508004870602550256C2567256825642565255925F5
S315080048805825522553256B256A2518250C25882574
S3150800489084258C2590258025B103DF009303C0036A
S315080048A0A303C303B500C403A6039803A903B4036B
S315080048B01E22C603B50329226122B100652264229D
S315080048C020232123F7004822B0001922B7001A2214
S315080048D07F20B200A025A00000600008002000008C
S315080048E0030000000080000800200000040000000B
S315080048F000A00008002000000500000000C0000815
S31508004900002000000600000000E00008002000006B
S315080049100700000000000108002000000800000051
S3150800492000200108002000000900000000400108DE
S31508004930002000000A0000000060010800200000B6
S315080049400B00000000800108002000000C00000099
S3150800495000A00108002000000D00000000C00108AA
S31508004960002000000E00000000E001080020000002
S315080049700F000000809A90418E418F804545454939
S3150800498049498E8F9092924F994F555559999A9BAE
S315080049909C9D9E9F41494F55A5A5A6A7A8A9AAAB28
S315080049A0AC21AEAFB0B1B2B3B4B5B6B7B8B9BABB4D
S315080049B0BCBDBEBFC0C1C2C3C4C5C6C7C8C9CACBB1
S315080049C0CCCDCECFD0D1D2D3D4D5D6D7D8D9DADBA1
S315080049D0DCDDDEDFE0E1E2E3E4E5E6E7E8E9EAEB91
S315080049E0ECEDEEEFF0F1F2F3F4F5F6F7F8F9FAFB81
S315080049F0FCFDFEFF433A5C576F726B5C736F66741F
S31508004A00776172655C4F70656E424C545C54617296
S31508004A106765745C44656D6F5C41524D434D335F09
S31508004A2053544D33325F4F6C696D65785F53544DFF
S31508004A303332503130335F4941525C426F6F745C98
S31508004A406D61696E2E630000433A5C576F726B5C4A
S31508004A50736F6674776172655C4F70656E424C540D
S31508004A605C5461726765745C536F757263655C410B
S31508004A70524D434D335F53544D33325C4941525C7A
S31508004A80766563746F72732E63000000433A5C5751
S31508004A906F726B5C736F6674776172655C4F706575
S31508004AA06E424C545C5461726765745C536F7572E0
S31508004AB063655C41524D434D335F53544D33325C0D
S31508004AC0756172742E630000433A5C576F726B5CB3
S31508004AD0736F6674776172655C4F70656E424C548D
S31508004AE05C5461726765745C536F757263655C6666
S31508004AF0696C652E6300000050617273696E6720E9
S31508004B006669726D776172652066696C6520746F77
S31508004B10206F627461696E206572617365207369BE
S31508004B207A652E2E2E0000004669726D77617265D1
S31508004B302075706461746520737563636573736645
S31508004B40756C6C7920636F6D706C657465640A0D9D
S31508004B50000000004F70656E696E67206669726DA9
S31508004B60776172652066696C6520666F722072656A
S31508004B706164696E672E2E2E000000004669726D0C
S31508004B8077617265207570646174652072657175E8
S31508004B906573742064657465637465640A0D000042
S31508004BA05374617274696E67207468652070726FD9
S31508004BB06772616D6D696E672073657175656E6381
S31508004BC0650A0D0052656164696E67206C696E65D9
S31508004BD02066726F6D2066696C652E2E2E455252C0
S31508004BE04F520A0D00000000496E76616C69642018
S31508004BF0636865636B73756D20666F756E642E2EBC
S31508004C002E4552524F520A0D00000000CBE9FFFF15
S31508004C10400F000004000020000000005FD4FFFFE2
S31508004C200400000018010000000000200000000039
S31508004C302F64656D6F70726F675F6F6C696D6578ED
S31508004C405F73746D3332703130332E73726563005F
S31508004C502062797465732066726F6D206D656D6F5D
S31508004C6072792061742030780000000057726974E8
S31508004C70696E672070726F6772616D20636865631D
S31508004C806B73756D2E2E2E002062797465732074F1
S31508004C906F206D656D6F7279206174203078000021
S31508004CA0436C6F73696E67206669726D77617265AA
S31508004CB02066696C650A0D0001030507090E1012C6
S31508004CC01416181C1E00000050726F6772616D6D15
S31508004CD0696E6720000000002F626F6F746C6F6743
S31508004CE02E7478740000000080B540210148FEF754
S31508004CF067FB01BD484A0008222A3A3C3E3F7C7FB2
S31508004D000000000045726173696E672000000000AC
S31508004D10C046C046C046C046FFF724FA2B2C3B3D8A
S31508004D205B5D00004552524F520A0D004F4B0A0D6B
S31508004D30000000004F70656E424C540001000000F0
S70508004D1194
